:100000000C942A000C9445000C9445000C94450077
:100010000C9445000C9447000C9445000C9445004A
:100020000C9445000C9445000C9445000C9445003C
:100030000C9445000C9445000C9445000C9445002C
:100040000C9445000C9445000C9445000C9445001C
:100050000C94450011241FBECFE5D4E0DEBFCDBF18
:1000600010E0A0E6B0E0E0EEFAE002C005900D92EC
:10007000A837B107D9F710E0A8E7B0E001C01D929A
:10008000AC37B107E1F70C946B000C9400001F92A1
:100090000F920FB60F9211242F933F938F939F933C
:1000A00086B597B52091780030917900821B930B2B
:1000B00090937B0080937A0086B597B590937900F2
:1000C000809378009F918F913F912F910F900FBE59
:1000D0000F901F901895CEE4D4E0DEBFCDBFEE2484
:1000E000FF248FEF87BB88BB0E94880160E0862FCA
:1000F0000E947C0180E88FBD81E08EBDFDBCECBC20
:1001000080E289BF789480E690E00E94E80140E0B8
:100110005AE560E070E029E030E0CA010197F1F7AC
:100120002150304037FFF9CF88B390E8892788BB4A
:1001300080917A0090917B008E159F0541F37C01A0
:1001400060E081E00E94C20180917A0090917B0082
:100150009C014427552760E070E488E390E00E940A
:100160004E053F932F9381E790E09F938F9381E11A
:1001700090E09F938F938E010F5F1F4F1F930F93FC
:100180000E940902C8010E94E8018DB79EB7089637
:100190000FB6F8949EBF0FBE8DBFB9CF8150F0F758
:1001A000089581509040E8F708951F938AB38E60B8
:1001B0008ABB8AB38F708ABB8BB3846F8BBBDB988F
:1001C00082E00E94CE00D99A81E00E94CE0019B34D
:1001D000107FD99882E00E94CE00D99A81E00E94D7
:1001E000CE0089B382958F70182BD998812F9927CB
:1001F0001F9108951F938AB38E608ABB8AB38F7054
:100200008ABB8BB38C6F8BBB82E00E94CE00D99AE5
:1002100081E00E94CE0019B3107FD99882E00E943D
:10022000CE00D99A81E00E94CE0089B382958F706A
:10023000182BD998812F99271F9108950E94D500D6
:100240008823E4F3089582E00E94CE00D99A81E0E9
:100250000E94CE00D99808950F931F93082F0E94F3
:100260001E018AB38E6F8ABB11E08BB381238BBBD7
:10027000902F907F8BB3892B8BBB0E9423018BB374
:1002800081238BBB802F992724E0880F991F2A9503
:10029000E1F72BB3282B2BBB0E9423011F910F9159
:1002A00008950F931F93082F0E941E018AB38E6F2B
:1002B0008ABB11E08BB381238BBB902F907F8BB3D4
:1002C000892B88608BBB0E9423018BB381238BBB5E
:1002D000802F992734E0880F991F3A95E1F72BB3C7
:1002E000282B28602BBB0E9423011F910F9108959A
:1002F00081E00E942C010895882319F08EE090E09F
:1003000002C08CE090E0611101960E942C010895DA
:100310001F938AB38E6F8ABB80E096E30E94D10060
:1003200011E08BB381238BBB8BB380638BBB0E94AB
:10033000230182EC9EE00E94D1000E9423018CE503
:1003400090E00E94D1000E9423018CE590E00E9481
:10035000D100DC980E9423018CE590E00E94D1003E
:1003600088E20E942C0186E00E942C010E94780104
:10037000612F812F0E947C011F91089582E00E94CD
:100380002C010895823050F4603140F48295880F3A
:10039000880F807C860F80580E942C0108950E944F
:1003A0001E010E94D500992746E0969587954A95AB
:1003B000E1F799278170907008950E941E010E94B4
:1003C000D50099278F73907008950E945101089568
:1003D000CF93DF93EC018881882331F089910E94CB
:1003E000E50188818823D1F7DF91CF910895CF93DC
:1003F000DF93EC01FC0121968491882339F00E945F
:10040000E501FE01219684918823C9F7DF91CF9100
:1004100008950F931F93CF93DF93CDB7DEB72E9739
:100420000FB6F894DEBF0FBECDBF0D891E892F8990
:10043000388D698D7A8D86E08C831A83098337FF26
:1004400005C08FEF9FE79E838D8304C0215030400D
:100450003E832D83AE01455E5F4FCE0101960E9423
:100460004502ED81FE818E179F070CF4FC01E00F21
:10047000F11F10822E960FB6F894DEBF0FBECDBFCF
:10048000DF91CF911F910F9108952F923F924F923C
:100490005F926F927F928F929F92AF92BF92CF9214
:1004A000DF92EF92FF920F931F93CF93DF93CDB71D
:1004B000DEB762970FB6F894DEBF0FBECDBFEE2455
:1004C000FF2487011C017E876D872A01CC24DD244F
:1004D000FC01D782C682838181FD68C28FEF9FEFC6
:1004E00078C28D859E8501969E878D87C0FE4BC202
:1004F0008F8580538A30D0F49F85903339F46620FD
:1005000029F4C3FC03C0E0E0F1E08DC08AE0689EFE
:10051000602C1124FF856F0E20ED620E67FE02C075
:100520005FE7652EC3FC42C2762C40C2C3FE04C006
:10053000662011F441E0642EEF858E2F992787FD08
:100540009095883691058CF5853691050CF06EC036
:100550008335910509F493C084359105CCF48B3231
:10056000910509F449C08C3291054CF48032910513
:1005700009F446C08332910509F44AC0FEC18D32A8
:10058000910509F440C08E32910509F444C0F5C1CB
:100590008336910509F450C0843691050CF08AC069
:1005A0008835910509F4BCC0E8C18037910509F48C
:1005B000B1C08137910584F48C36910591F18D3667
:1005C00091052CF48936910509F474C0D6C18F3693
:1005D000910509F49CC0D1C18537910509F4A2C0E9
:1005E0008637910524F48337910571F1C6C18837A8
:1005F000910509F495C0C1C180E190E0C82AD92ACB
:10060000E0E2F0E010C080E890E0C82AD92ACEC12C
:10061000E0E4F0E008C088E090E0C82AD92A662427
:10062000C5C1E4E0F0E0CE2ADF2AC0C13FE3E32EFB
:100630007A94F3E6FF873CC1F20182E090E0480E35
:10064000591EE0807A9434C1F20182E090E0480EB5
:10065000591EA081B1817D01C3FE09C0862D992755
:1006600087FD9095BC01CD010E9416051FC0FD01BC
:1006700001900020E9F73197EA1BE88B18C0F201DE
:1006800082E090E0480E591E0190F081E02D7F013C
:10069000C3FE09C0862D992787FD9095BC01CF0127
:1006A0000E940B0503C0CF010E940205888B988928
:1006B000791AFEC0C2FE0AC0F20184E090E0480E42
:1006C000591E20813181428153810CC0F20182E0A8
:1006D00090E0480E591E808191819C01442737FD8E
:1006E0004095542F79018A0157FF0CC0E2E0F0E0F9
:1006F000CE2ADF2A10950095F094E094E11CF11CBD
:10070000011D111D8FEB9FEFC822D92227C098E051
:10071000988B08C0E0E4F0E0CE2ADF2AF8E7FF87F4
:1007200020E1288BC2FE0AC0F20184E090E0480E6E
:10073000591E20813181428153810AC0F20182E039
:1007400090E0480E591E808191819C0144275527D5
:1007500079018A01EFECFFEFCE22DF22CE01019674
:100760009A8B898B9889892E9924AA24BB24C80145
:10077000B701A50194010E944E05DC01CB01E98976
:10078000FA8980838A3024F0FF858F0F815201C05F
:10079000805DE989FA898193FA8BE98BC801B701F9
:1007A000A50194010E944E0579018A0121153105A8
:1007B00041055105E1F6E98881E090E08C0F9D1F2D
:1007C000E81AC60182739070892B09F07A94C6FEEC
:1007D0000DC0872D992787FD9095E889E03121F498
:1007E0002EEF722E780E02C0782E7A94C3FE0FC0C0
:1007F000262D332727FD30958E2D992782179307B5
:100800002CF087EF9FEFC822D92201C06E18C3FEDB
:1008100002C0761801C07E18C60180789170892BBD
:1008200051F4872D7A94181634F4B10180E290E0E7
:100830000E942105F6CFC1FE04C0B1018DE290E017
:100840000BC0C4FE04C0B1018BE290E005C0C5FE40
:1008500005C0B10180E290E00E942105C6FE10C0F3
:10086000B10180E390E00E9421059889903141F424
:10087000B101EF858E2F992787FD90950E94210564
:10088000D0FE0AC0872D7A94181634F4B10180E3A3
:1008900090E00E942105F6CFC3FE0AC0862D6A941F
:1008A000181634F4B10180E390E00E942105F6CFE0
:1008B00090E8B92EBC2051F4872D7A94181634F4A0
:1008C000B10180E290E00E942105F6CFFF85F3366A
:1008D00041F48E2DB101992787FD90950E94210545
:1008E00040C02F852337B1F488898150888B8F3F92
:1008F000C1F1F70180810894E11CF11CB101992735
:1009000087FD90950E94210598899150988B9F3F73
:1009100081F727C0EF85E33579F4F889F150F88B3A
:10092000FF3FF9F0F7018491B10199270E94210559
:100930000894E11CF11CF1CF6E010894C11CD11C7C
:1009400089899A898C159D0561F0E989FA898291D6
:10095000FA8BE98BB101992787FD90950E942105BB
:10096000EFCFBB2069F0872D7A9418164CF4B101B3
:1009700080E290E00E942105F6CFB1010E9421059E
:10098000CC24DD2413C09F85953241F481E0C82E2C
:10099000D12C6624762CEAE0E88B08C0B101FF85F3
:1009A0008F2F992787FD90950E942105F101838162
:1009B00083FF04C0ED85FE85F49103C0ED85FE85BF
:1009C000F081FF872F85222309F08BCDF1018681ED
:1009D000978162960FB6F894DEBF0FBECDBFDF9150
:1009E000CF911F910F91FF90EF90DF90CF90BF902C
:1009F000AF909F908F907F906F905F904F903F90BF
:100A00002F900895FC0105900020E9F780959095BE
:100A10008E0F9F1F0895FC010590615070400110DA
:100A2000D8F7809590958E0F9F1F0895FC01615017
:100A3000704001900110D8F7809590958E0F9F1F00
:100A400008950F931F93CF93DF938C01EB018B815C
:100A5000992781FF1CC082FF0DC02E813F818C81B0
:100A60009D812817390764F4E881F9810193F9839E
:100A7000E88306C0E885F985802F0995892B39F42C
:100A80008E819F8101969F838E83C80102C08FEF64
:100A90009FEFDF91CF911F910F910895A1E21A2E40
:100AA000AA1BBB1BFD010DC0AA1FBB1FEE1FFF1F12
:100AB000A217B307E407F50720F0A21BB30BE40B62
:100AC000F50B661F771F881F991F1A9469F76095A9
:100AD0007095809590959B01AC01BD01CF01089563
:100AE0004465206672657175656E74696520697309
:080AF0000025347520487A004E
:00000001FF
